:0200000039289D
:08000800FF0003088301FE0064
:100010000408FD00592883178001840AFF3E031D50
:100020000C283428A301A200FF30A207031CA30759
:10003000031C34280330A100DF3020201428A10144
:10004000E83EA000A109FC30031C2928A0070318E2
:100050002628A0070000A10F262820182F28A01C62
:100060003328000033280800831383120313000091
:10007000080007309F00C0308316860010308500CE
:100080008113203084005D3083120C20A030840066
:1000900050300C202030840030300B2083160112A9
:1000A000811681158B160B11CE30831281008B17B0
:1000B0008D280B11CE308100AA0A3C302A02031D84
:1000C0008628AA01A80A0A302802031D8628A8014A
:1000D000A70A06302702031D8628A60AA801A70141
:1000E000043026020130031D0030A4000230250236
:1000F0000130031D0030240503198028A601A50145
:100100000A302602031D8628A601A50A7D08840060
:100110007E088300FF0E7F0E0900A501A601A7013E
:10012000A8018316851183128515280886000130E1
:1001300012208316851183128511860132301F200B
:100140008316051183120515270886000130122039
:100150008316051183120511860132301F20831684
:10016000851083128514260886000130122083161C
:10017000851083128510860132301F2083160510EA
:1001800083120514250886000130122083160510FD
:1001900083120510860102301220CF2091280130F1
:1001A000061B0301A40001302918030124050319CB
:1001B000E828A80A0A302802031DE628A801A70A91
:1001C00006302702031DE628A801A7012914F328F9
:1001D0000301061B0130A400030129180130240586
:1001E0000319F32829100130861B0301A4000130F4
:1001F000A9180301240503190C29A60A0A302602AE
:10020000031D0A29A601A50A06302502031D0A2995
:10021000A601A501A91417290301861B0130A4001A
:100220000301A9180130240503191729A910080092
:040230006300182926
:02400E00503F21
:00000001FF
